:0200000480007A
:100000006F000005732F2034930F80006308FF03F7
:10001000930F90006304FF03930FB0006300FF038E
:10002000130F000063040F0067000F00732F2034CC
:1000300063540F006F00400093E19153171F0000BD
:1000400023223FFC171F000023200FFC6FF01FFF2F
:100050009300000013010000930100001302000050
:100060009302000013030000930300001304000038
:100070009304000013050000930500001306000020
:100080009306000013070000930700001308000008
:10009000930800001309000093090000130A0000F0
:1000A000930A0000130B0000930B0000130C0000D8
:1000B000930C0000130D0000930D0000130E0000C0
:1000C000930E0000130F0000930F0000732540F102
:1000D0006310050097020000938202017390523072
:1000E000735044749702000093820201739052305F
:1000F00073500018970200009382420273905230AE
:100100009B021000939252039382F2FF7390023B82
:100110009302F0017390023A73504030970200004E
:1001200093824201739052307350203073503030BC
:100130009301000097020000938202ED7390523009
:10014000130510001315F501635C05000F00F00F97
:10015000930110009308D005130500007300000000
:1001600093020000638A020073905210B7B200003D
:100170009B8292107390223073500030372500001C
:1001800073200530735030009702000093824201C3
:1001900073901234732540F173002030172400004F
:1001A000130444E69301200007310400273824009B
:1001B000033504019B031000939373029383F31799
:1001C000939373016318750893013000073104009D
:1001D00027282400033504019B0310009393730226
:1001E0009383F3179393730163167506930140008D
:1001F0000721040027282400033504019B03100075
:10020000939373029383F3179393730163147504A9
:10021000930150000731840027382400033504017E
:100220009B0310F89393130293831310939363012A
:1002300063127502930160000721840027382400AF
:10024000033504019B0310D093936301631475007D
:10025000631030020F00F00F6380010093911100D2
:1002600093E111009308D00513850100730000008D
:100270000F00F00F930110009308D0051305000044
:1002800073000000731000C00000000000000000B8
:10029000000000000000000000000000000000005E
:1002A000000000000000000000000000000000004E
:0C02B00000000000000000000000000042
:1010000000000000000000000000000000000000E0
:1010100000000000000000000000000000000000D0
:1010200000000000000000000000000000000000C0
:1010300000000000000000000000000000000000B0
:081040000000000000000000A8
:10200000000080BF0000004000004040000080C091
:10201000EFBEADDEBEBAFECAEA1DADAB0DD03713C2
:040000058000000077
:00000001FF
